:100000009E0A1C02100F43071A0A7C00F207130A0B
:100010001D021E0143070E0A7100170AFD009D0212
:100020004306FE00170AF90C3D00060C3E001102C3
:100030002600250ABC021C029401430646041C0249
:1000400095014307250A06042604E106250AE20C69
:1000500021000008010966062F0A01092B0A560C27
:1000600030000109F0004306390A01096606320A28
:100070009C0A0109F20C330001096607460A0109CE
:100080006607460A0109F3023D0A9C0A0109040CAD
:10009000300066064E0A0109B002490A01090B0C3C
:1000A000900003079C0A01096607590A0109B0027A
:1000B000540A01093F0C900003069C0A01091A0228
:1000C0002400100220000109060C300066066B0AAD
:1000D0000109B002660A01090D0C900003079C0A91
:1000E00001096607760A0109B002710A01093F0C8D
:1000F000900003069C0A01090109060C30006606FF
:10010000840A0109B0027F0A01090D0C900003075F
:100110009C0A010966078F0A0109B0028A0A0109CF
:100120003F0C900003069C0A01091B0224001002E8
:1001300020000109F2040008F2052A0A25006600E1
:10014000080C0600080C0200E20C2100F90C3D002E
:10015000060C3E007000740075003E0C39007C00F7
:1001600072007100170C3A00160C3B0001092A09B5
:1001700001091204320401091802F70101090304FC
:100180003703010917023800280C97000306CD0A2F
:10019000010912052A0CB700770201092B0C970000
:1001A0000307D60A01093205290CB7000109030427
:1001B00057033500010901091902F6010109030479
:1001C00036030109160239000109210C96000306C5
:1001D000EC0A01095204F10A01095205200C9600AB
:0A01E0003400010912023100B60AD2
:021FFE00EB0FE7
:00000001FF
